 dvfc_mc34704

 Timestamp is 4da293a7 (Mon Apr 11 17:37:43 2011)

 Preferred load address is 10000000

 Start         Length     Name                   Class
 0001:00000000 00000004H .CRT$XCA                CODE
 0001:00000004 00000004H .CRT$XCZ                CODE
 0001:00000008 00000004H .CRT$XIA                CODE
 0001:0000000c 00000004H .CRT$XIZ                CODE
 0001:00000010 00000004H .CRT$XPA                CODE
 0001:00000014 00000004H .CRT$XPZ                CODE
 0001:00000018 00000004H .CRT$XTA                CODE
 0001:0000001c 00000004H .CRT$XTZ                CODE
 0001:00000020 00000098H .rdata                  CODE
 0001:000000b8 00000029H .rdata$debug            CODE
 0001:000000e4 00001088H .text                   CODE
 0001:0000116c 00000048H .xdata                  CODE
 0001:000011b4 00000050H .idata$2                CODE
 0001:00001204 00000014H .idata$3                CODE
 0001:00001218 0000008cH .idata$4                CODE
 0001:000012a4 000000ceH .idata$6                CODE
 0001:00001380 00000098H .edata                  CODE
 0002:00000000 0000008cH .idata$5                DATA
 0002:00000090 00000064H .data                   DATA
 0002:000000f4 0000005cH .bss                    DATA
 0003:00000000 00000128H .pdata                  DATA

  Address         Publics by Value              Rva+Base       Lib:Object

 0000:00000000       ___safe_se_handler_count   00000000     <absolute>
 0000:00000000       ___safe_se_handler_table   00000000     <absolute>
 0001:00000000       __xc_a                     10001000     corelib0:crt0init.obj
 0001:00000004       __xc_z                     10001004     corelib0:crt0init.obj
 0001:00000008       __xi_a                     10001008     corelib0:crt0init.obj
 0001:0000000c       __xi_z                     1000100c     corelib0:crt0init.obj
 0001:00000010       __xp_a                     10001010     corelib0:crt0init.obj
 0001:00000014       __xp_z                     10001014     corelib0:crt0init.obj
 0001:00000018       __xt_a                     10001018     corelib0:crt0init.obj
 0001:0000001c       __xt_z                     1000101c     corelib0:crt0init.obj
 0001:0000003c       ??_C@_1CA@DNJNIIBE@?$AAI?$AAN?$AAT?$AAR?$AA_?$AAE?$AAV?$AAE?$AAN?$AAT?$AA_?$AAD?$AAV?$AAF?$AAC?$AA?$AA@ 1000103c     dvfc_common_topaz_v1:dvfc.obj
 0001:0000005c       ??_C@_1M@EENNDIOJ@?$AAI?$AAn?$AAd?$AAe?$AAx?$AA?$AA@ 1000105c     dvfc_common_topaz_v1:dvfc.obj
 0001:00000068       ??_C@_1CE@KCPPCGKP@?$AAE?$AAV?$AAE?$AAN?$AAT?$AA_?$AAD?$AAV?$AAF?$AAC?$AA_?$AAW?$AAO?$AAR?$AAK?$AAE?$AAR?$AA?$AA@ 10001068     dvfc:dvfc.obj
 0001:0000008c       ??_C@_1BO@ICEODACO@?$AAE?$AAV?$AAE?$AAN?$AAT?$AA_?$AAS?$AAE?$AAT?$AAP?$AAO?$AAI?$AAN?$AAT?$AA?$AA@ 1000108c     dvfc:dvfc.obj
 0001:000000ac       ??_C@_1M@LCEEOPDH@?$AAI?$AA2?$AAC?$AA1?$AA?3?$AA?$AA@ 100010ac     pmicsdk:mc34704sdk.obj
 0001:000000e4       DvfcInitVoltageSupplies    100010e4 f   voltctrl.obj
 0001:0000013c       DvfcConvertVoltage         1000113c f   voltctrl.obj
 0001:000001c8       DvfcUpdateSupplyVoltage    100011c8 f   voltctrl.obj
 0001:00000274       DVF_Deinit                 10001274 f   dvfc_common_topaz_v1:dvfc.obj
 0001:00000278       DVF_Open                   10001278 f   dvfc_common_topaz_v1:dvfc.obj
 0001:0000027c       DVF_Close                  1000127c f   dvfc_common_topaz_v1:dvfc.obj
 0001:0000028c       DVF_IOControl              1000128c f   dvfc_common_topaz_v1:dvfc.obj
 0001:00000470       DVF_Init                   10001470 f   dvfc_common_topaz_v1:dvfc.obj
 0001:000005d4       BSPDvfcGetThreadPriority   100015d4 f   dvfc:dvfc.obj
 0001:000005e4       DvfcMapDevPwrStateToSetpoint 100015e4 f   dvfc:dvfc.obj
 0001:0000061c       BSPDvfcGetSupportedDx      1000161c f   dvfc:dvfc.obj
 0001:00000624       BSPDvfcPowerGet            10001624 f   dvfc:dvfc.obj
 0001:00000640       BSPDvfcPowerSet            10001640 f   dvfc:dvfc.obj
 0001:000006b4       DvfcUpdateSetpoint         100016b4 f   dvfc:dvfc.obj
 0001:00000910       BSPDvfcIntrServ            10001910 f   dvfc:dvfc.obj
 0001:0000095c       BSPDvfcInit                1000195c f   dvfc:dvfc.obj
 0001:00000a78       BSPDvfcDeinit              10001a78 f   dvfc:dvfc.obj
 0001:00000a80       DisableThreadLibraryCalls  10001a80 f   coredll:COREDLL.dll
 0001:00000a90       SetLastError               10001a90 f   coredll:COREDLL.dll
 0001:00000aa0       WaitForSingleObject        10001aa0 f   coredll:COREDLL.dll
 0001:00000ab0       InterruptDone              10001ab0 f   coredll:COREDLL.dll
 0001:00000ac0       CeSetThreadPriority        10001ac0 f   coredll:COREDLL.dll
 0001:00000ad0       CreateThread               10001ad0 f   coredll:COREDLL.dll
 0001:00000ae0       InterruptInitialize        10001ae0 f   coredll:COREDLL.dll
 0001:00000af0       KernelIoControl            10001af0 f   coredll:COREDLL.dll
 0001:00000b00       CreateEventW               10001b00 f   coredll:COREDLL.dll
 0001:00000b10       RegCloseKey                10001b10 f   coredll:COREDLL.dll
 0001:00000b20       RegQueryValueExW           10001b20 f   coredll:COREDLL.dll
 0001:00000b30       OpenDeviceKey              10001b30 f   coredll:COREDLL.dll
 0001:00000b40       EventModify                10001b40 f   coredll:COREDLL.dll
 0001:00000b50       QueryPerformanceFrequency  10001b50 f   coredll:COREDLL.dll
 0001:00000b60       QueryPerformanceCounter    10001b60 f   coredll:COREDLL.dll
 0001:00000b70       MmMapIoSpace               10001b70 f   ceddk:CEDDK.dll
 0001:00000b80       DDKClockSetpointRequest    10001b80 f   cspddk:CSPDDK.dll
 0001:00000b90       DDKClockSetpointRelease    10001b90 f   cspddk:CSPDDK.dll
 0001:00000ba0       DDKClockLock               10001ba0 f   cspddk:CSPDDK.dll
 0001:00000bb0       DDKClockUnlock             10001bb0 f   cspddk:CSPDDK.dll
 0001:00000bc0       DDKClockGetSharedConfig    10001bc0 f   cspddk:CSPDDK.dll
 0001:00000bd0       PmicOpen                   10001bd0 f   pmicsdk:mc34704sdk.obj
 0001:00000c14       PmicSetRegister            10001c14 f   pmicsdk:mc34704sdk.obj
 0001:00000ca8       PmicGetRegister            10001ca8 f   pmicsdk:mc34704sdk.obj
 0001:00000d44       PmicRegulatorSetVoltageLevel 10001d44 f   pmicsdk:mc34704sdk.obj
 0001:00000d80       PmicRegulatorGetVoltageLevel 10001d80 f   pmicsdk:mc34704sdk.obj
 0001:00000de0       DllMain                    10001de0 f   corelib0:dllmain.obj
 0001:00000eec       _DllMainCRTStartup         10001eec f   corelib0:pegdmain.obj
 0001:00000fd8       _cexit                     10001fd8 f   corelib0:cexit.obj
 0001:00000fe8       _initterm                  10001fe8 f   corelib0:crt0dat.obj
 0001:00001014       _cinit                     10002014 f   corelib0:crt0dat.obj
 0001:00001074       __security_init_cookie     10002074 f   corelib0:seccinit.obj
 0001:000010c0       __crt_ExitProcess          100020c0 f   corelib0:exitproc_proxy.obj
 0001:000010cc       __C_specific_handler       100020cc f   corelib1:COREDLL.dll
 0001:000010dc       memset                     100020dc f   corelib1:COREDLL.dll
 0001:000010ec       __rt_sdiv64by64            100020ec f   corelib1:COREDLL.dll
 0001:000010fc       _XcptFilter                100020fc f   corelib1:COREDLL.dll
 0001:0000110c       free                       1000210c f   corelib1:COREDLL.dll
 0001:0000111c       __security_gen_cookie2     1000211c f   corelib1:COREDLL.dll
 0001:0000112c       TerminateProcess           1000212c f   coredll:COREDLL.dll
 0001:0000113c       I2COpenHandle              1000213c f   i2csdk:I2CSDK.dll
 0001:0000114c       I2CTransfer                1000214c f   i2csdk:I2CSDK.dll
 0001:0000115c       I2CSetFrequency            1000215c f   i2csdk:I2CSDK.dll
 0001:000011b4       __IMPORT_DESCRIPTOR_COREDLL 100021b4     coredll:COREDLL.dll
 0001:000011c8       __IMPORT_DESCRIPTOR_CEDDK  100021c8     ceddk:CEDDK.dll
 0001:000011dc       __IMPORT_DESCRIPTOR_CSPDDK 100021dc     cspddk:CSPDDK.dll
 0001:000011f0       __IMPORT_DESCRIPTOR_I2CSDK 100021f0     i2csdk:I2CSDK.dll
 0001:00001204       __NULL_IMPORT_DESCRIPTOR   10002204     coredll:COREDLL.dll
 0002:00000000       __imp_MmMapIoSpace         10003000     ceddk:CEDDK.dll
 0002:00000004       \177CEDDK_NULL_THUNK_DATA  10003004     ceddk:CEDDK.dll
 0002:00000008       __imp_WaitForSingleObject  10003008     coredll:COREDLL.dll
 0002:0000000c       __imp_InterruptDone        1000300c     coredll:COREDLL.dll
 0002:00000010       __imp_CeSetThreadPriority  10003010     coredll:COREDLL.dll
 0002:00000014       __imp_CreateThread         10003014     coredll:COREDLL.dll
 0002:00000018       __imp_InterruptInitialize  10003018     coredll:COREDLL.dll
 0002:0000001c       __imp_KernelIoControl      1000301c     coredll:COREDLL.dll
 0002:00000020       __imp_SetLastError         10003020     coredll:COREDLL.dll
 0002:00000024       __imp_RegCloseKey          10003024     coredll:COREDLL.dll
 0002:00000028       __imp_RegQueryValueExW     10003028     coredll:COREDLL.dll
 0002:0000002c       __imp_OpenDeviceKey        1000302c     coredll:COREDLL.dll
 0002:00000030       __imp_EventModify          10003030     coredll:COREDLL.dll
 0002:00000034       __imp_QueryPerformanceFrequency 10003034     coredll:COREDLL.dll
 0002:00000038       __imp_QueryPerformanceCounter 10003038     coredll:COREDLL.dll
 0002:0000003c       __imp_CreateEventW         1000303c     coredll:COREDLL.dll
 0002:00000040       __imp_DisableThreadLibraryCalls 10003040     coredll:COREDLL.dll
 0002:00000044       __imp___security_gen_cookie2 10003044     corelib1:COREDLL.dll
 0002:00000048       __imp_free                 10003048     corelib1:COREDLL.dll
 0002:0000004c       __imp___C_specific_handler 1000304c     corelib1:COREDLL.dll
 0002:00000050       __imp_memset               10003050     corelib1:COREDLL.dll
 0002:00000054       __imp___rt_sdiv64by64      10003054     corelib1:COREDLL.dll
 0002:00000058       __imp__XcptFilter          10003058     corelib1:COREDLL.dll
 0002:0000005c       __imp_TerminateProcess     1000305c     coredll:COREDLL.dll
 0002:00000060       \177COREDLL_NULL_THUNK_DATA 10003060     coredll:COREDLL.dll
 0002:00000064       __imp_DDKClockUnlock       10003064     cspddk:CSPDDK.dll
 0002:00000068       __imp_DDKClockLock         10003068     cspddk:CSPDDK.dll
 0002:0000006c       __imp_DDKClockSetpointRelease 1000306c     cspddk:CSPDDK.dll
 0002:00000070       __imp_DDKClockSetpointRequest 10003070     cspddk:CSPDDK.dll
 0002:00000074       __imp_DDKClockGetSharedConfig 10003074     cspddk:CSPDDK.dll
 0002:00000078       \177CSPDDK_NULL_THUNK_DATA 10003078     cspddk:CSPDDK.dll
 0002:0000007c       __imp_I2CTransfer          1000307c     i2csdk:I2CSDK.dll
 0002:00000080       __imp_I2CSetFrequency      10003080     i2csdk:I2CSDK.dll
 0002:00000084       __imp_I2COpenHandle        10003084     i2csdk:I2CSDK.dll
 0002:00000088       \177I2CSDK_NULL_THUNK_DATA 10003088     i2csdk:I2CSDK.dll
 0002:00000090       g_DvfcIrq                  10003090     dvfc:dvfc.obj
 0002:000000ec       __security_cookie          100030ec     corelib0:seccinit.obj
 0002:000000f0       __security_cookie_complement 100030f0     corelib0:seccinit.obj
 0002:0000013c       _exitflag                  1000313c     corelib0:cexit.obj
 0002:00000140       g_pCRM                     10003140     <common>
 0002:00000144       __onexitend                10003144     <common>
 0002:00000148       __onexitbegin              10003148     <common>
 0002:0000014c       _pRawDllMain               1000314c     <common>

 entry point at        0001:00000eec

 Static symbols

 0001:00000428       DvfcIntrServThread         10001428 f   dvfc_common_topaz_v1:dvfc.obj
 0001:00000784       DvfcWorkerThread           10001784 f   dvfc:dvfc.obj
 0001:00000dfc       _DllMainCRTStartupHelper   10001dfc f   corelib0:pegdmain.obj
 0001:00000f18       doexit                     10001f18 f   corelib0:cexit.obj
